:020000040000FA
:0600000000308A002C28EC
:10000800FC0003088301DE0083128C1E18288C1262
:1000180006161808DD001A08DD00981C15281812A5
:1000280018165D08A00026280B1D262886150B111A
:0800380064308100A70A2808CA
:100040002702031C2628A701AB14861183125E0821
:100050008300FC0E7C0E0900203084005E303420CA
:10006000392804068001840A0406031D312864002F
:100070000034F9230630831686000A308312A80064
:100080008322640044236400832043288401700891
:10009000F8007108F9007208FA007308FB00F20119
:1000A000F301F001F1010310FB0CFA0CF90CF80C50
:1000B000031C68287408F00775080318750FF1070A
:1000C00076080318760FF20777080318770FF307FF
:1000D000780879047A047B04031974280310F40D5A
:1000E000F50DF60DF70D5328840803190034730835
:1000F00080008403720880008403710880008403F8
:10010000700880000034EB23031C8C282008733A0D
:10011000031D822B4423822BF023031C98280030DC
:100120006121F22201306121AB140230AB060800DC
:100130002008CF00A0010612C22800306121DA2376
:10014000B62800306121D323B62800306121E02396
:10015000B628003061212021031CB028A60AAB2854
:10016000A60302306121F22A042282230130612990
:10017000A8030130280203180800A801A80A0800F3
:10018000A80A08004F0803190800203A0319A928F3
:10019000443A0319C028023A0319B8280C3A031943
:1001A0009D28013A0319A128073A0319A5281E3AE8
:1001B0000319B428013A031D0800442B8312CA080E
:1001C000031DE628D101D10AD201C9236D30F40004
:1001D0004E30F500C630F6004130F7004B08F00015
:1001E0004C08F1004D08F2004E08F300462039306B
:1001F000F4003030F500F601F70174087007F800DC
:100200007108F90075080318750FF9077208FA00EC
:1002100076080318760FFA077308FB0077080318AF
:10022000770FFB077808CB007908CC007A08CD005F
:100230007B08CE00F1004D08F0007F30F10508008A
:100240008312D201D1015108D5005208B323031CF7
:10025000552951082507D000D01F30290310080068
:100260005008803A763E031C372903100800260800
:10027000F000F101F01BF1035208F0070318F10A36
:100280007108803AF200803072021830031970024F
:10029000031C4C29031008005008D60026085207FA
:1002A000BC22031C552903100800D10A0430510256
:1002B000031C2329D20A04305202031C22290314EE
:1002C00008008312D000D40126085407D200183049
:1002D000520203189329D30125085307033ED10086
:1002E0000D30510203188A295308D5005408B3234E
:1002F000031C8A295108D50052089B23500B8229E0
:10030000483089295008023A031D88295830892924
:1003100020306523D30A04305302031C6C29D50115
:10032000D50A01309B23D40A043054020318080074
:1003300064298312A10EF030A105A20EA205A30E1E
:10034000A305A40EA405D001D1015108043E5623F3
:10035000F1005008D82271050319B4295008033C54
:100360005623D2005108A022D10A04305102031CA6
:10037000A529D00A0430500203180800A4298312CA
:10038000D200D4015208D500D5080319D729540842
:10039000D6005503BC22003003180130D3005408A6
:1003A000D6005308D7005508E221D50BC7295408B9
:1003B000D600D7010030E221D40A0A3054020318D3
:1003C0000800C2298312D8000A30F1005808F00052
:1003D0000310F00C0310F00C0310700C8F23560761
:1003E000D900580807395623DA00D708031DFE291B
:1003F00059082C3E84005A098005080059082C3EF3
:1004000084005A0880040800F523D4010230D50086
:1004100054089B237C306523D3015308D60054082D
:10042000BC220318152A2030162A5830D200652322
:10043000D30A0A305302031C0D2A7C306523D40AE8
:100440001830540203180800062A8312D300F00063
:10045000F03E0318FF34103E031CFF3402308A00C4
:100460003530700703188A0A820006346034063477
:1004700060340E344034443444340C346034063434
:10048000C0340E3420340E3480348312D301260855
:100490005307D100D20125085207D0005208D500D9
:1004A0005308B323031C5A2A5008D600D701D70A91
:1004B0005108E221D20A04305202031C4B2AD30A0B
:1004C0000430530203180800472A8312D100510751
:1004D0002522D200F039F000F00E0F30F005700840
:1004E000A10052080F39A2000314510D2522D20099
:1004F000F039F000F00E0F30F0057008A30052083C
:100500000F39A400080083168614061183120615FD
:100510008316181219309900181518171814831219
:1005200018138C1283168C168312981718160B1733
:100530008B1683168112811101308312810008000D
:100540008312D300AF2A5208A10408005208A20463
:1005500008005208A30408005208A4040800530825
:100560000319A32A013A0319A62A033A0319A92A4F
:10057000013A031D0800AC2A8312D9000A30F100A9
:100580005908F0000310F00C0310F00C0310700C6D
:100590008F235607D700590807395623D800570824
:1005A0002C3E8400000858050310031D03140800A6
:1005B0008312D800E42A2108E22A2208E22A23082A
:1005C000E22A2408D900F02A58080319DB2A013A44
:1005D0000319DD2A033A0319DF2A013A0319E12A34
:1005E000590808008312A60A2021031808002608CB
:1005F000803A7D3E031CAB15A603023061214522E3
:100600000923A6010430A500A90AE623AA0A01309D
:1006100061298312D001D10151083223031C152B0B
:10062000D001D00A5108BF21A90AD10A18305102BD
:10063000031C0C2BD008031908000422822B831200
:10064000D101D0015008D600D7015108E221D00ACB
:100650000A305002031C222BD10A18305102031811
:100660000800212B8312D200D3015308D600520870
:10067000BC2203183D2B03100800D30A0A30530292
:10068000031C352B031408008B1374231F2304222F
:10069000A6010430A500E623AA01AA0AA901A70120
:1006A000AB01AB0AA0018B17013061298312DB007B
:1006B0000130F0005B08F100F10A602B0310F00D2F
:1006C000F10B5E2B7008DC0008008312D700990044
:1006D000831698168312D80106130617D80AFA3023
:1006E0005802031808006C2B1B3065235B30652310
:1006F0003F306523323065236C3065231B30652322
:100700006630652B28308312D50014309B232908CE
:10071000A723203065230030A7232A08A72BF00049
:100720000030711870070310F00D0310F10CF10880
:1007300003190800912B8312D6001B306523593012
:1007400065235608203E65235508203E652B8312FD
:10075000D200520E0F39D300BE23652352080F3941
:10076000D300BE23652B8312D600D822D7005508AC
:10077000562357050310031D031408008312D400E9
:100780000A30540254080318C72B303E0800573E65
:10079000080083125108CB005208CC00CD01CE01D5
:1007A000CA01CA0A080099212021031808009921CA
:1007B000992199298312A5032021031CA50A080069
:1007C0008312A50A2021031CA5030800DE2070085F
:1007D0000739D000652A03108312AB1903140800EF
:1007E00003108312AB18031408001B306523483034
:0A07F000652B8B018B1783120800A4
:02400E00A93FC8
:00000001FF
